:020000040000FA
:1000000003138316113085000F30860083120130F0
:100010009800FF309700851499018C01051E0D286A
:1000200000008C0F0E288F011010051A15280F30B4
:100030008C008C0B1928051A002808308D000F3011
:100040008C008C0B2128101D3828151C2E28051219
:1000500083160130850083120000352805168316AB
:1000600011308500831200000000950C0A303928F9
:100070000E308C008C0B3A288E0C8E13051E8E17BA
:10008000000000008D0B1F280E308C008C0B4628C2
:10009000101D522805168316113085008312101189
:1000A0000B3053280E308C008C0B5428051E002872
:1000B0008F0A0F030739820764286A286B286C2887
:1000C0006D28742875287628901C692813089500D7
:1000D0001015152815281528152804300E020319A7
:1000E0008514031D85101528152815288F01212139
:1000F00090198620940B81280130940090101011E3
:10010000852812089500901410150D2896000F39B7
:100110008207D028C1289E289928DF28E4289E2815
:100120009928CB28C628A828A328B728BC28B228F5
:10013000AD2828309200003093001E29283092000C
:10014000103093001E2928309200353093001E296C
:1001500028309200373093001E29283092000E304C
:1001600093001E29283092001E3093001E2928304B
:100170009200473093001E292830920045309300AA
:100180001E2928309200413093001E292830920009
:10019000513093001E29183092002B3093001E29F5
:1001A000183092005E3093001E29183092003230D1
:1001B00093001E2918309200323093001E29183007
:1001C0009200333093001E2985141E30A5000515BA
:1001D000072105110D21A50BE7280130A5001921E4
:1001E000A50BEF28FF30A5000515012105110D21F4
:1001F000A50BF42885101E290D30A000A00BFE28A9
:1002000008001B30A300FC20A30B032908001A30B0
:10021000A100FC20A10B09290800C830A400FC2083
:10022000A40B0F290800C830A400FC20A40B15293A
:1002300008000530A2000D21A20B1B2904309400F8
:1002400008009011991C2C2925290518332999108B
:10025000053096009015BB29051C332999140430EC
:1002600096009015BB29E0308600000000000609CA
:100270000F3903194429960016187A2996187D29F2
:100280001619802996198329D030860000000000B5
:1002900006090F390319552996001618862996184C
:1002A000892916198C2996198F29B03086000000EB
:1002B000000006090F3903196629960016189229BD
:1002C000961895291619982996199B297030860039
:1002D0000000000006090F39031977299600161847
:1002E0009E299618A1291619A4299619A729101232
:1002F000FF30AA2910120030AA2910120130AA29B1
:1003000010120230AA2910120330AA291012043048
:10031000AA2910120530AA2910160630AA2910168B
:100320000730AA2910120830AA2910120930AA2968
:1003300010160A30AA2910160B30AA2910160C30F4
:10034000AA2910160D30AA2910160E30AA29101647
:100350000F30AA29960017020319B829980BBB2958
:100360000330980016089700FF3C031D9015BB2929
:0A037000101EBB29901516080800A6
:02400E00F93F78
:00000001FF
